:020000040800F2
:100000007023002049010008D9060008D506000821
:10001000D7060008D10600086107000800000000AC
:10002000000000000000000000000000FD060008C5
:10003000D306000800000000FB060008FF060008C9
:100040006301000863010008630100086301000800
:1000500063010008630100086301000863010008F0
:1000600063010008630100086301000863010008E0
:1000700063010008630100086301000863010008D0
:1000800063010008630100086301000863010008C0
:1000900063010008630100086301000863010008B0
:1000A00063010008630100086301000863010008A0
:1000B0006301000863010008630100086301000890
:1000C0006301000863010008630100086301000880
:1000D0006301000863010008630100086301000870
:1000E0006301000863010008630100086301000860
:1000F0006301000863010008630100086301000850
:10010000630100086301000863010008630100083F
:10011000630100086301000863010008630100082F
:10012000630100086301000863010008630100081F
:10013000DFF810D000F02CFA004800478D1C0008B2
:10014000AFF3008070230020064880470648004730
:10015000FEE7FEE7FEE7FEE7FEE7FEE7FEE7FEE777
:10016000FEE7FEE7050700083101000800F0004245
:1001700030F000400AD0C10D01F56071C0F31600E7
:1001800042EA0151C208400711437047002001466E
:10019000704730B50B46014600202022012409E0BB
:1001A00021FA02F59D4205D303FA02F5491B04FA30
:1001B00002F52844151EA2F10102F1DC30BD2DE943
:1001C000F05F0546002092469B46884606468146DB
:1001D00040241BE0284641464746224600F0F9F9F4
:1001E00053465A46C01A914110D31146184622462A
:1001F00000F0E0F92D1A67EB01084F462246012076
:10020000002100F0D7F917EB00094E41201EA4F1A0
:100210000104DFDC484631462A464346BDE8F09FEC
:100220002DE9FE4F804681EA0300C00F0C46009086
:1002300021F0004123F00045B8EB0200A94105D2AE
:100240004046214690461C460B46024623F000409D
:10025000104347D0270DC7F30A00C3F30A51029099
:10026000401A019040286BDAC3F3130040F4801B5E
:100270000098924620B10023D2EB030A63EB0B0BEC
:1002800001985946C0F14002504600F093F90646E5
:100290000D4650465946019A00F0ABF910EB0800A4
:1002A0006141002487EA115284EAE7731A4340D07F
:1002B000009A62B3019A012A4FEA075215DC001B2B
:1002C00061EB02014FF0004202EA0752CDE9004221
:1002D000001C41F5801132462B4600F0ABF903B00B
:1002E000BDE8F08F40462146F9E7001B61EB0201B3
:1002F000001C41F5801300185B412018A2F500177F
:1003000047EB030140EAD570B6196D4111E06D0865
:100310004FEA360645EAC0754FEA0752001B61EB0B
:100320000201001C41F5801149084FEA3000001914
:10033000514132462B4603B0BDE8F04F00F06BB997
:100340000098012240000023D0EB020263EBE0732F
:10035000009821464FEAE074B8EB000061EB04011D
:10036000E9E783F000435BE781F0004158E72DE9BE
:10037000FE4F81EA030404F0004421F000410094A0
:100380004FF0000B23F0004350EA01045ED052EA24
:1003900003045BD0C3F30A54C1F30A552C44A4F2FE
:1003A000F3340194A0FB0254C1F3130141F4801112
:1003B000C3F3130343F4801301FB024400FB034E19
:1003C000840A970A44EA815447EA8357A4FB0768E2
:1003D00002958D0A05FB07854FEA932C04FB0C540C
:1003E0002705029D4FEA065847EA1637B5EB080580
:1003F0006EEB070C870E920E47EA811742EA8312D2
:10040000A7FB0201B6EB0B0164EB00042B0D43EAE2
:100410000C335E1844EB1C50DA465146E7FB0201F0
:10042000C5F313044FEA0B3343EA14534FEA043283
:10043000019C43EA0603A4F10C040294009CCDE95C
:1004400000B400F0F7F803B0BDE8F08F00200146DB
:10045000F9E72DE9F04D81EA030404F0004B21F0A7
:10046000004514464FF0000A23F0004150EA05020F
:1004700020D054EA01021DD0C5F30A570246C5F345
:100480001303C1F31300C1F30A5640F4801543F47B
:100490008013A7EB0608101BD64608F2FD3873EB55
:1004A000050002D308F1010801E092185B41B8F1A0
:1004B000000F03DA00200146BDE8F08D00204FF464
:1004C0008011064684460EE0171B73EB050705D323
:1004D000121B63EB050306434CEA010C49084FEA83
:1004E000300092185B4150EA0107EDD152EA030057
:1004F00012D082EA040083EA0501084305D0101BEC
:10050000AB4106D20122002306E000224FF0004357
:1005100002E06FF0010253101AEB06004CEB085199
:1005200010EB0A0041EB0B01BDE8F04D00F073B891
:10053000C1F30A52C1F3130140F2FF3341F48011B9
:100540009A4202DA00200146704740F233439A4251
:10055000A2F2334202DC524200F03BB800F02AB86B
:1005600030B5041E71F1000404DB4FF0004440423A
:1005700064EB0101141E73F1000405DB1C464FF00F
:100580000043524263EB0403994208BF904230BDDE
:10059000064C074D06E0E06840F0010394E80700D0
:1005A00098471034AC42F6D3FFF7C6FDA8630008A5
:1005B000C8630008202A04DB203A00FA02F1002078
:1005C00070479140C2F1200320FA03F31943904091
:1005D0007047202A04DB203A21FA02F000217047FC
:1005E00021FA02F3D040C2F120029140084319469B
:1005F0007047202A06DBCB17203A41FA02F043EA83
:10060000E07306E041FA02F3D040C2F120029140CB
:1006100008431946704710B5141E73F1000408DA38
:10062000401C41F1000192185B411A4301D120F0B6
:10063000010010BD2DE9F04D92469B4611B1B1FA73
:1006400081F202E0B0FA80F220329046FFF7B2FF6A
:1006500004460F4640EA0A0041EA0B0153465A4657
:10066000084313D0114653EA010019D0C8F14002E3
:100670005046FFF7AEFF05460E46504659464246E5
:10068000FFF798FF084305D0012004E020463946D3
:10069000BDE8F08D0020054346EAE0762C43374361
:1006A0000A986305E40AA0EB08000022FD0A44EA68
:1006B00047540A3002D500200146E9E70105101928
:1006C0006941DDE9084500196941BDE8F04DA2E73F
:1006D000FEE77047FEE7FEE770470907090E0028AE
:1006E00006DA00F00F0000F1E02080F8141D7047DA
:1006F00000F1E02080F8001470477047704700F068
:1007000009BE0000134882B0016841F47001016025
:100710001148016841F001010160416841F0800128
:100720004160002144F620620091009B5B1C009315
:100730009342FAD34160C1620168084A11400160E6
:100740004FF41F018160016821F48021016002B033
:1007500001F052BE88ED00E000100240FFFFF6FEFF
:10076000FEE700000FB4054B10B503A9044A029838
:1007700000F00CF910BC5DF814FB0000591A0008D9
:10078000180000200FB4084B10B504A902AA039862
:1007900000F0FCF8044602A9002000F07AFC204694
:1007A00010BC5DF814FB00009310000802E008C8BC
:1007B000121F08C1002AFAD170477047002001E0DB
:1007C00001C1121F002AFBD17047000070B5074C11
:1007D00005460221204601F0E9FD0028F9D029460E
:1007E0002046BDE8704001F0C0BD00000038004068
:1007F00010B5044C8021204601F0D8FD0028F9D125
:1008000010BD0000003800402DE9FF5F82B00021DC
:10081000DDE90430020DDDF840B0034318D044F6A2
:100820001050A2F2FF3242431514119801281FD034
:10083000A5EB0B00401C5FEA000A4FF000064E4F8C
:10084000DFF83891B046504615D5CAF1000413E0E0
:10085000119801244AA3012801D16FEA0B010298E3
:10086000119AC0E90031C0E9024206B0BDE8F09F2C
:10087000CBF10000DFE704460021404A491842EB73
:100880000450CDE9001012E0E00707D032463B46A5
:1008900040464946FFF76BFD8046894632463B4657
:1008A00010461946FFF763FD06460F466410002CFC
:1008B000EAD1DDE90401DDE90023BAF1000F06DA2F
:1008C000FFF755FD42464B46FFF751FD05E0FFF7A8
:1008D000C0FD42464B46FFF7BCFD04460E460022D3
:1008E000284BFFF73DFE03D84FF0FF30014607E0ED
:1008F0000022254B20463146FFF792FCFFF718FEF9
:10090000102409E0002C0ADB0A220023FFF757FC21
:10091000039B30321A55641E50EA0102F2D1641C66
:10092000039AC4F111031444119A012A03D001223D
:1009300008430DD10AE0084304D000204FF0110B0A
:10094000119072E7A3EB0B056D1E0DE05B4504DD16
:100950004FF0000205F1010504E003DA4FF0000258
:10096000A5F10105002AECD002981199C0E90231E5
:10097000C0E9004579E70000000014400000F03FA6
:10098000300000000000F0430000E03F2DE9FF4F81
:1009900095B09A46884606460025EEE1252877D18F
:1009A00000242746F94A0121039400E0044316F885
:1009B000013F203B01FA03F01042F7D130782A289A
:1009C00011D06FF02F033078A0F13002092A16D829
:1009D000039A44F0020402EB820203EB4202104449
:1009E000761C0390EFE758F8042B0392002A03DAF1
:1009F000504244F40054039044F00204761C3078D2
:100A00002E2816D116F8010F44F004042A280DD020
:100A10006FF02F023078A0F13003092B09D807EBD3
:100A2000870302EB4303C718761CF3E758F8047BEF
:100A3000761C30786C280FD006DC4C2817D068283C
:100A40000DD06A2814D104E0742810D07A280FD170
:100A50000DE044F400140AE044F4801401E044F48E
:100A600040147278824202D104F58014761C761C00
:100A7000307866280BD013DC582877D009DC0028A2
:100A800075D04528F6D04628F4D047281AD193E1EE
:100A900018E0632835D0642879D0652812D18BE11D
:100AA000702873D008DC6728F1D069286FD06E28D1
:100AB0000DD06F2806D1ACE073282CD0752874D0E7
:100AC000782853D05246179990476D1C54E1C4F3CF
:100AD0000250022809D003280DD0D8F800100428AD
:100AE0000DD00D6008F1040846E1D8F80010EA17AF
:100AF000C1E90052F6E7D8F800100D80F2E70D705A
:100B0000F0E718F8041B8DF8001000208DF80100A4
:100B1000EB46012003E058F804BB4FF0FF306107BB
:100B20004FF0000102D40DE009F101018946B942FC
:100B30000FDA8145F8DB1BF809100029F4D108E031
:100B400009F1010189468142FADB1BF809100029ED
:100B5000F6D103985346A0EB090721463846179A69
:100B600000F080FA284400EB090507E044E008E1C2
:100B70000DE01BF8010B524617999047B9F1010996
:100B8000F7D2534621463846179AF2E039E00A2157
:100B9000C4F302524FF0000B0091022A06D058F81D
:100BA000040BC117032A09D00AE023E008F107006B
:100BB00020F00702F2E80201904605E000B2C117FA
:100BC000042A01D140B2C117002906DA0A460021E1
:100BD000404261EB02012D2202E0220504D52B22C6
:100BE0008DF80420012203E0E20701D02022F7E77C
:100BF000914657E00A2100E010214FF0000B0091D0
:100C00000BE010214FF0000B44F004040827009182
:100C100003E008204FF0000B0090C4F30252022AB8
:100C200005D058F8040B0021032A08D008E008F189
:100C3000070020F00702F2E80201904603E080B2CC
:100C4000042A00D1C0B24FF0000922072AD5327819
:100C5000702A07D0DDF800C08CF0100C5CEA0B0C99
:100C600005D00EE040228DF80420012208E050EA71
:100C7000010306D030238DF804308DF805200222C0
:100C80009146009B83F0080353EA0B030AD150EA14
:100C9000010201D1620705D530228DF804204FF002
:100CA00001097F1E3278582A04D039A20C920CAA6E
:100CB00002920BE03BA2F9E75B46009AFFF77FFA4E
:100CC0000C9B9B5C029A521E0292137050EA010226
:100CD000F2D1029804A9081A00F1200B600702D58E
:100CE00024F4803400E001275F4502DDA7EB0B0010
:100CF00000E0002000EB0B01009003984944401AEB
:100D00000390E00306D453462146179A039800F057
:100D1000A9F90544002706E001A85246C05D1799CD
:100D200090476D1C7F1C4F45F6DBE0030CD5534606
:100D30002146179A039800F095F9054404E0302005
:100D40005246179990476D1C0099481E0090002943
:100D5000F5DC08E00298029952460078491C02919D
:100D6000179990476D1CBBF10001ABF1010BF1DC51
:100D70005BE100F065F90544761C307800287FF4CB
:100D80000DAE19B02846BDE8F08F0000092801001B
:100D900030313233343536373839616263646566F1
:100DA00000000000303132333435363738394142B3
:100DB0004344454600000000600700D4062708F1C0
:100DC000070020F00700F0E80223804603F0004C03
:100DD0005FEA0C0001D097A009E0200501D596A09C
:100DE00005E0E00701D095A001E0AFF24C001390C0
:100DF000307823F0004365280CD006DC452809D064
:100E000046281DD047287FD13BE0662818D06728A8
:100E10007AD136E00021112F01DB112000E0781C8F
:100E2000CDE9000104A90CA8FFF7EEFCDDE90D01F6
:100E30000C9A4FF0000B07F10109109200914EE05F
:100E40004FF000400097CDE9011004A90CA8FFF76E
:100E5000DBFCDDE90D020C9B0F994FF0000B914676
:100E60001093009211B9791C00EB0109B7EB09004E
:100E700003D4C0F1FF3B07F10109A9EB0700019082
:100E800042E0012F00DA01270021112F01DD11209E
:100E900000E03846CDE9000104A90CA8FFF7B4FC36
:100EA000DDE90D010C9A00914FF0000BB94610924C
:100EB00021070FD4009A4A4503DA914601E0A9F1CF
:100EC0000109B9F1010F05DD109AA9F10101515C89
:100ED0003029F4D0B84202DA10F1040F03DA01210C
:100EE000CDE9011010E0002803DC8344A9EB0001E8
:100EF00002E0411C494500DD8946A0EB0B00401C87
:100F000001904FF000400290200705D40198484519
:100F100002DB4FF0FF30019000208DF84B0002986B
:100F20000DF14B07B0F1004F25D002200C902B2083
:100F30000D90029800280CDA404202902D200D906E
:100F400007E00A210298FFF724F93031029007F8F0
:100F5000011D0C99481E0C900029F2DC0298002813
:100F6000EFD1791E0D980870307800F0200040F025
:100F7000450007F8020D11A8C01BC01D0290139870
:100F8000007800B1012000EB0901019801EBE0714C
:100F9000029801440398401A401E0390E00306D4CF
:100FA00053462146179A039800F05CF805441398BD
:100FB000007818B15246179990476D1CE00323D56D
:100FC00053462146179A039800F04CF805441BE05D
:100FD000BBF1000F07DB0098584504DD1098179906
:100FE00010F80B0001E01799302052469047019805
:100FF0000BF1010B401E05F10105019004D12E20DB
:101000005246179990476D1CB9F10001A9F10109E9
:10101000DEDC05E017F8010B5246179990476D1C6E
:101020000299481E02900029F4DC53462146179A83
:1010300003989EE62D0000002B0000002000000019
:101040002DE9F041044600251E461746880404D4C5
:1010500005E039462020B0476D1C641EF9D52846AE
:10106000BDE8F0812DE9F041044600251E4690467A
:10107000C80301D5302700E02027880404D505E007
:1010800041463846B0476D1C641EF9D52846BDE878
:10109000F0810A68531C0B6010707047816841F042
:1010A0000801816081680907FCD4816841F004016E
:1010B000816081684907FCD470471205A2F580124F
:1010C00001290BD0022908D1816B21F440118163E1
:1010D00002F44011826B114381637047C16A21F4AD
:1010E0007001C16202F47001C26A1143C1627047AB
:1010F00010B540F2096001F009F9012001F054F83F
:101100001D4C01221102204600F0C1F800220221EC
:10111000204600F0BCF84FF4E0420221204600F0E7
:101120005AF8002000F09AF80021204600F026F836
:10113000022211462046FFF7C0FF0723102200219C
:10114000204600F063F8072311220121204600F019
:101150005DF801220221204600F022F800F0C0F8DC
:10116000204600F015F8012000F0CAF82046BDE83E
:101170001040FFF793BF0000002401400029816860
:1011800002D041F4006101E021F400618160704708
:101190008168C90703D1816841F00101816070470E
:1011A000002A4FEAC1720AD01AB1826842F4801252
:1011B000826089070ED5816841F4004109E01AB1C7
:1011C000826822F480128260890703D5816821F445
:1011D000004181607047012909D0022906D1816848
:1011E00021F4E0418160816811438160704781682A
:1011F00021F46021F6E702688A43026070470246E4
:10120000002012680A4200D00120704730B5846B7C
:10121000C4F30155846B491BC91C01EB81011F25D7
:101220008D40AC4302FA01F12143816307240A2A6D
:1012300008D2016902EB42029440A14393400B4360
:10124000036130BD122AFCD2C1680A3A02EB4202A5
:101250009440A14393400B43C36030BD04490A68E6
:1012600022F470220A600A6802430A607047000094
:1012700004240140CA0703D0826842F480028260DD
:10128000890703D5816841F4001181607047002A05
:101290004FEAC15211D0002A03DA426842F4807248
:1012A00042604A0503D5426842F480624260890781
:1012B00015D5816841F0020110E0002A03DA426886
:1012C00022F4807242604A0503D5426822F48062AB
:1012D0004260890703D5816821F00201816070476F
:1012E0000248016841F40001016070470824014090
:1012F00002494A6802434A6070470000002004E047
:1013000003490A6810440A688242FCD3704700000F
:101310001000002002480168491C0160704700006D
:101320001000002070B5054D29680C1802E000205F
:1013300000F02EFF2868A042F9D370BD10000020F5
:1013400000224FF48051014800F0A0BB000C014086
:1013500001221103014800F099BB0000000C01407C
:1013600000224FF48041014800F090BB000C014086
:1013700001229103014800F089BB0000000C0140EC
:101380002DE9F04700258A468146FA264FF01008DD
:101390002946284600F0E8FA242000F03DFBFFF73C
:1013A000CFFF00275FF0000419F80500FFF70EFAE1
:1013B000641C6D1CB442F7D37F1C4745F2D3FFF782
:1013C00017FAFFF7C5FF0021084600F0CDFA2620E6
:1013D00000F022FB0025FFF7B3FF00275FF00004B9
:1013E0001AF80500C043C0B2FFF7F0F9641C6D1C89
:1013F000B442F5D37F1C4745F0D3FFF7F9F9FFF767
:10140000A7FFBDE8F04700F0CCBA10B504461020A5
:1014100000F002FB2046BDE8104000F0E1BA10B534
:1014200000F092FA3220FFF76BFF00F095FA3220BD
:10143000FFF766FF00F0C3FA002858D1122000F031
:10144000EBFA00F0BCFA002851D1012000F0E4FAD8
:10145000272000F0C5FA012000F0C2FA012000F0B8
:10146000BFFA112000F0D8FA012000F0B9FA4420A8
:1014700000F0D2FA002000F0B3FA0F2000F0B0FA2A
:10148000452000F0C9FA272000F0AAFA012000F058
:10149000A7FA002000F0A4FA002000F0A1FA3C20F6
:1014A00000F0BAFA052000F09BFA212000F0B4FA0F
:1014B000002000F095FA802000F092FA182000F049
:1014C000ABFA802000F08CFA4E2000F0A5FA002044
:1014D00000F086FA4F2000F09FFA272000F080FAF3
:1014E000012000F07DFA00F06AFA002800D0012007
:1014F00010BD000010B588B040F2026000F006FF99
:1015000040F2036000F002FF4FF4C06000F0FEFE06
:10151000234C4FF4807303221021204600F01EFB61
:101520004FF4004303224821204600F017FB1D4CD6
:101530004FF4804303221021204600F00FFB4FF4AC
:10154000204303221821204600F008FBA3140322A5
:101550001021204600F002FB40F20E7000F0D6FE93
:10156000114C204600F004FF684600F03BFF4FF4AA
:10157000404001904FF482700090032000210590BC
:101580006015CDE9021018200491069069462046A6
:1015900000F011FF204600F0E3FE08B010BD00008F
:1015A00000080140000C01400038004010B54FF425
:1015B0000041034800F025FB002800D0012010BDA9
:1015C0000008014030B500210A4AC3B20DE00020F6
:1015D00006E000BF01FB04041568401C80B22B55D7
:1015E000148A8442F6D8491C89B2508A8842EED8BF
:1015F00030BD00005C1F00202DE9F84F1F469146CA
:1016000082468846151A01D5A0EB09057C1A002CE4
:1016100000DDCC1B4FF0FF32CA4501D2012000E0B3
:1016200010460090B84500D2012293462E1941463B
:1016300050460A9A00F018F8B4EB460F07DCCA458A
:1016400010D0009926440AEB01001FFA80FAB5EB8E
:10165000460FECDBB84505D008EB0B002E441FFA13
:1016600080F8E4E7BDE8F88F491E401E89B280B2D9
:1016700000F052B82DE9F8418046DDE907501E46DA
:1016800017460C4648B90CE023463A4619464046F0
:101690000095FFF7B1FF641CA4B2B442F4D3BDE8D7
:1016A000F8810B4640460095FFF7A6FF42463346B9
:1016B000214610460095FFF79FFF3A4623463146E4
:1016C00010460095FFF798FF3346424619463846C4
:1016D0000095FFF791FFE2E730B50B4C039D2060CA
:1016E00021816281A5814D074FEAD10000D0401CC5
:1016F00020826282E38123B1B42B02D0A180E280F8
:1017000030BDA280E18030BD5C1F0020014908602F
:10171000704700005C1F002070B5184C2346E68916
:101720001B89D6B125465A2E6D891AD0B42E1DD0EC
:10173000B6F5877F10D103460846218A25684143C4
:1017400001EBD3018020002A6C5C03F0070220FA31
:1017500002F010D02043685470BD591A491E8BB254
:10176000EBE7181A401E83B2681A01E00B46281AEC
:10177000401E80B2E1E784436C5470BD5C1F0020C2
:101780002DE9FC4F401C1FFA80F9491C1C468DB204
:10179000A9EB0400AB46CDF80490FA285FDC082CD6
:1017A0000ED0600700D0012000EBD400610810FBD0
:1017B00001F080B28246203A90B2009000204BE0C7
:1017C0000620F7E7082C12D00C2C17D0102C1AD0BA
:1017D000182C44D10098244900EBC00001EB800193
:1017E000002711F80860F00712D00B9A13E0009858
:1017F0001E4900EB400001EB4001F1E700981C4955
:1018000000EB4000EAE71B49009801EB0011E7E715
:101810000B9830B3002229464846FFF725FF6D1C80
:101820007F1C7608BFB2ADB2082FDCD309F10100EE
:101830001FFA80F9082C0BD00198A9EB0000B0EB3F
:10184000540F05D10BF10800DDF804901FFA80FB5E
:1018500008F101005D4680B280465045B2D3BDE834
:10186000FC8F0122D7E700002452000898450008A9
:10187000C0470008344C00082DE9FF4F401C82B0DF
:101880004FF0000984B2491CCDE9009492468DB214
:101890004A46AB46580700D0012000EBD300059024
:1018A00010462FE0002026E00F98002610F809705F
:1018B00009F101001FFA80F9F8072BD0109838B30E
:1018C000002229462046FFF7CFFE6D1C761C7F08BC
:1018D000B6B2ADB2082EEFD3641C0198A4B2211A9F
:1018E000514504D10BF10800019C1FFA80FB08F15F
:1018F00001005D4680B280465045D5D30098401C1B
:1019000080B2009005998842CCD306B0BDE8F08F34
:101910000122D6E7109AD4E72DE9F8411E46144675
:1019200088460546079F09E033464146284600970A
:10193000FFF726FF05EB560085B2641C2278002ACB
:10194000F2D1BDE8F881000000224FF48071014817
:1019500000F09CB80008014001221102014800F08B
:1019600095B800000008014070B5C0F3C705F9291B
:1019700001D92E2403E0A1F22711484284B24E205F
:1019800000F04AF8284600F02BF84F2000F044F809
:10199000E0B200F025F8C4F30020BDE8704000F08C
:1019A0001FB810B5222000F037F8F72000F018F823
:1019B000202000F031F8BDE81040AFF3008070B592
:1019C000002444F6206506E0641CAC424FF00100A0
:1019D00005D8FFF795FCFFF7E9FD0028F4D170BDAD
:1019E00010B50446FFF7ACFC21460A4C204600F037
:1019F000BCFC0221204600F0D9FC0028F9D080214F
:101A0000204600F0D3FC0028F9D1BDE81040FFF7D4
:101A10009FBC00000038004010B50446FFF7A0FC52
:101A2000FFF78EFC21460B4C204600F09EFC022165
:101A3000204600F0BBFC0028F9D08021204600F0B1
:101A4000B5FC0028F9D1FFF783FCBDE81040FFF793
:101A50008FBC00000038004070B5074D0446C1B28D
:101A6000284600F0ADFD0721284600F0DEFD0028E5
:101A7000F9D0204670BD00000038014001480068E0
:101A80007047000010000020416170470AB10161F9
:101A9000704741617047000010B54FF4C06000F01E
:101AA00035FC40F2026000F031FC40F2036000F0CF
:101AB0002DFC01210A4800F0AFF801230322282160
:101AC000084800F04BF8084C04230322102120465C
:101AD00000F044F82046BDE810400421FFF7D4BFD1
:101AE0000002300000080140000C014010B5194C04
:101AF0002115031B4A00A04221D009DC164BC01857
:101B000017D0884218D0904222D14FF4417408E097
:101B10008B4217D0934218D0B3F5406F18D14FF4D1
:101B20004274204600F00EFC2046BDE8104000F054
:101B3000FBBB40F20234F4E740F20334F1E740F239
:101B40000534EEE740F20634EBE740F20734E8E70D
:101B500010BD00000014014000F8FEBF2DE9F04365
:101B600001F00F04CD0602D5042A19D01443002534
:101B70004FF00F095FF0010202FA05F61E401AD07D
:101B800007684FEA850C09FA0CF827EA080704FAF7
:101B90000CF848EA0708282908D0482908D008E0A6
:101BA000C26B44F003041A43C263E0E7466100E0FD
:101BB0000661C0F800806D1CADB2082DDCD308258D
:101BC00002FA05F61E4016D047684FEA8508A8F1CC
:101BD000200809FA08FC27EA0C0704FA08FC4CEA7A
:101BE000070C282902D0482902D002E0466100E013
:101BF0000661C0F804C06D1CADB2102DE0D3BDE885
:101C0000F0838068084000D001207047C068084019
:101C100000D0012070470000F0B5144C002801DA14
:101C2000E36900E06368420D120185B2C0F3015719
:101C30009540C0F30346032F05D0C2020AD5032204
:101C4000B240934307E023F0E062636823F0E0636F
:101C5000636002E0AB4343F0E06201B12A43002835
:101C600001DAE261F0BD6260F0BD000000000140F9
:101C70000168054A1140B1F1005F04D14168006874
:101C800080F30888084770470000FE2F88B000F0F6
:101C9000B5FA0720FFF72CFB00F00CFCFFF7FCFE69
:101CA000FFF726FA00F02EFC0127FFF7E7FE0646B5
:101CB0003546B2A0FEF756FDB7A0FEF753FDBDA016
:101CC000FEF750FDC3A0FEF74DFDC8480168C8A04F
:101CD000FEF748FD012000F099FA0146C8A0FEF782
:101CE00041FD022000F092FA0146C9A0FEF73AFD3C
:101CF000032000F08BFA0146C9A0FEF733FDCCA00B
:101D0000FEF730FDFFF7F6FBFFF789FB4FF0FF080A
:101D1000B423FA227A21CC48CDF80080FFF7DCFC0E
:101D2000B423FA227A21C948CDF80080FFF7D4FC09
:101D3000C548FFF7EBFCFF20FFF744FC0024C44834
:101D4000CDE900047A23FA2221462046FFF794FDCC
:101D5000BE48FFF7DBFCFF20FFF734FCBD49CDE9AF
:101D6000001800217A23FA220846FFF785FDB749BB
:101D7000B548FFF705FB4FF4FA50FFF7C1FAB24838
:101D8000FFF7C4FCFF20FFF71DFC1823B2A20021BF
:101D90000A200094FFF7C0FD1023B4A21D210A20E1
:101DA0000094FFF7B9FD1023B7A232210A20009456
:101DB000FFF7B2FDA548FFF7A9FCFF20FFF702FCE3
:101DC000B8A102A8FEF7DEFC182302AA47210A20C8
:101DD0000094FFF7A1FD4FF00108CDE900487423FE
:101DE000F02267210A20FFF745FC98499648FFF743
:101DF000C7FA0120FFF709FBDFF8B8A2DFF8B8B295
:101E0000DFF8B892FFF73AFEA8420AD9FFF736FE8C
:101E100000F5FA75012F4FF00401584615D0FFF771
:101E200033FEFFF72BFEB0420ED9FFF727FE00F17D
:101E30000A0601214846FFF7E4FE01289AF800103F
:101E400050466DD001290CD094E0FFF7DFFE012849
:101E500001D0012200E0002204215846FFF716FEBF
:101E6000DFE78AF80040012F01D0012700E00027BA
:101E700093A0FEF777FC02219748FFF7FBF902E0F9
:101E80000120FFF74FFA02219348FFF7B8F9002825
:101E9000F6D002219048FFF7AEF98F483C30006839
:101EA00040F6E4414843000B00EE100AB8EE400A49
:101EB000DFED8A0A30EEC00ADFED890A864880EE3F
:101EC000201AB3EE090A403031EE000A8AED020A08
:101ED0000068484300EE900AF8EE600A9FED811A10
:101EE00010EE100A60EE810ACAED030AFEF73EF911
:101EF00041EC100B7CA053EC102BFEF733FCDAF80E
:101F00000C00FEF733F941EC100B83A053EC102BBF
:101F1000FEF728FC39A0FEF725FCCAF8044029E0AA
:101F200009B980F800804168491CCAF804103229B8
:101F300020D38448006878B183A0FEF713FCBFF378
:101F40004F8F8048001D0168864A01F4E06111430B
:101F50000160BFF34F8FFEE783A0FEF703FC00F0A4
:101F6000C9FA5846FFF7C2FD4846FFF7BFFD87484C
:101F7000FFF77EFE002000F00BF943E70D0A5765DE
:101F80004163742053747564696F20436F726520D8
:101F9000426F6172640D0A007765616374737475D2
:101FA00064696F2E74616F62616F2E636F6D0D0ACD
:101FB00000000000776561637473747564696F2E47
:101FC000616C69657870726573732E636F6D0D0A4D
:101FD00000000000777777772E77656163742D7442
:101FE000632E636E0D0A0D0A00000000140000202D
:101FF00053797374656D436C6B3A25640D0A000068
:10200000434B5F4148422069732025640D0A00005C
:10201000434B5F415042312069732025640D0A0013
:10202000434B5F415042322069732025640D0A0002
:10203000457061706572204D6F64756C65205465E4
:1020400073740D0A000000001C000020BC0F00206B
:1020500058260008F8350008322E313320457061CB
:10206000706572204D6F64756C650000446573691E
:10207000676E65642042792057654163742053740C
:102080007564696F0000000077697468203235302C
:10209000207820313232207265736F6C7574696FED
:1020A0006E0000003E3E2048656C6C6F20576F72DA
:1020B0006C642E0000000020000C0140000801406C
:1020C00048656C6C6F2C576541637420537475645C
:1020D000696F0D0A000000000024014000C0B244F6
:1020E0009A998940000080395468652074656D7044
:1020F0006572617475726520646174612069732012
:1021000025322E31662064656772656573204365EC
:102110006C736975730D0A00546865207265666595
:1021200072656E636520766F6C74616765206461AB
:1021300074612069732025352E33666D56200D0A93
:102140000000000008ED00E0456E74657220494112
:102150005020426F6F746C6F61646572202E2E2E5A
:102160000D0A00000400FA05456E7465722073794B
:102170007374656D2049535020426F6F746C6F61AA
:10218000646572202E2E2E0D0A00000000F0FF1F45
:1021900004490A6822F004020A6008B120BF7047AF
:1021A00030BF704710ED00E0124A10B55168124B75
:1021B0001940D36A0C2823F0005317D2DFE800F04F
:1021C00006060606160916091010101041EA80319D
:1021D0000CE020F0040041EA803040F0805105E03E
:1021E00020F00C0041EA803143F000535160D3628B
:1021F00010BD000000100240FF3FFFEF0248416A9F
:1022000041F08071416270470010024070B537A5FF
:1022100088B02ECD8DE82E0035A20446D2E90012FA
:10222000CDE9041232A20020D2E90012CDE9061253
:10223000324A5168324BC1F3810119B1012901D0F1
:10224000022901D019462BE0516801F480352D494F
:10225000B5F5803F0AD1D56A15F0804F00D02A4BE2
:10226000556805F40035B5F5003F00D10B465168BF
:102270005568C1F383412D0101D541F01001556826
:102280006D0001D541F020010F2901D2891C06E023
:10229000A1F10F052F2D01D8491C00E03F21594322
:1022A0005368C3F303131DF8035021FA05F355686F
:1022B00004AEC5F302255268755D23FA05F5C2F335
:1022C000C22206AEB25C23FA02F244B1012C08D05D
:1022D000022C08D0032C00D1104608B070BD08466F
:1022E000FBE71846F9E72846F7E700000000000082
:1022F0000000000001020304060708090010024064
:1023000000127A0000093D00006CDC02054901EB77
:1023100090110A6800F01F030120984002430A60F0
:102320007047000000100240054901EB90110A6857
:1023300000F01F030120984082430A6070470000AC
:1023400000100240054901EB90110A6800F01F03DC
:102350000120984002430A607047000000100240CC
:10236000016841F0400101607047C16070470000A2
:102370000D4910B5401808D0B0F5806F08D0B0F501
:10238000784F0FD14FF4437404E040F20E4401E063
:1023900040F20F442046FFF7D5FF2046BDE810402D
:1023A000FFF7C2BF10BD000000C8FFBF8068084033
:1023B00000D001207047026802F441530A681A43B2
:1023C0004B6813438A681A43CB6813430A691A435C
:1023D0004B698969134319430160C16921F40061A4
:1023E000C16170470021016041608160C16041614D
:1023F00081610161704700002A480021026842F4AF
:10240000803202604FF6FF730268491C12F4003FED
:1024100001D19942F8D10168890300D4FEE7C1696E
:1024200041F08051C16120490A6842F440420A608B
:102430004268426042684260426842F480624260A0
:10244000426822F440324260426842F440324260C4
:102450004268164B1A4042604268154B1A4342606C
:10246000026842F08072026002689201FCD50A683C
:1024700042F480320A604A68D203FCD50A6842F40A
:1024800000320A604A689203FCD5416821F00301DA
:102490004160416841F00201416041680907FCD593
:1024A000704700000010024000700040FFFFC3B7FB
:1024B0000000340870B50E484FF47A710068B0FB24
:1024C000F1F0401EB0F1807F11D24FF0E024606146
:1024D00065170F212846FEF700F90020A0610720AC
:1024E00020612846BDE870400521FEF7F6B8FEE7FA
:1024F000140000204FF0E020002101614161816162
:102500007047000010B540F20260FFF7FFFE40F296
:102510000E60FFF7FBFE124C4FF4007303221821EC
:102520002046FFF71BFB2315032204212046FFF75B
:1025300015FB0C4C204600F047F84FF4E1312046E3
:1025400000F012F80421204600F07AF80821204615
:1025500000F07CF82046BDE8104000F061B80000B3
:10256000000801400038014070B5134B04460D4689
:102570000020E11A1A159C421BD005DC0F49611896
:1025800017D0914208D114E0914212D0B1F56C4FAE
:1025900002D10320FFF73AFE00EB5500B0FBF5F146
:1025A0004FF6F07201EA020001F00F010843A0604B
:1025B00070BD0220EEE70000004C004000BCFFBFF1
:1025C000C1F3080141607047134B10B5C21A1915C9
:1025D000984213D007DC114A80180CD088421AD1D7
:1025E00040F212440FE08A420BD0B2F56C4F12D188
:1025F00040F20E3407E040F2114404E040F213448C
:1026000001E040F214442046FFF79CFE2046BDE85E
:102610001040FFF789BE10BD004C004000BCFFBF5A
:10262000C16841F40051C160704700EB911000682F
:1026300001F01F0201219140084000D001207047A5
:10264000C26822F004020A43C2607047C26822F0E6
:1026500008020A43C260704700000000000000004A
:10266000000000000000000000000000000000006A
:10267000000000000000000000000000000000005A
:10268000000000000000000000000000000000004A
:10269000000000000000000000000000000000003A
:102C00008080808080800000000000C0E0E0E0E084
:102C1000C0C0000000000000000000000000000034
:102C200000000000000000000000000000000000A4
:102C30000000000000000000000000000000000094
:102C400000007EFEFEFEFEFEFE00000080FEFEFE98
:102C5000FEFEFEFEFC00000000FCFEFEFEFEFE3E50
:102C60000000000000000000808080808080000064
:102C70000000000000000000000080F8FEFEFEFEE4
:102C8000FEFEFEFEF08000000000000000000000DC
:102C9000000000808080808080000000000000F83C
:102CA000F8F8F8F8F8F80000000000000000000054
:102CB000000000000000E0F0F8FCFCFEFE7E7E3E1E
:102CC0003E7E7EFEFCFC783000000000F8F8F8F84C
:102CD000F8F8F8000000000000000000000000000C
:102CE00000000000000000000000000000000000E4
:102CF00000000000808080808000FFFFFFFFFFFF5A
:102D0000FF000000030F1F1F1F1F0F0F0000000018
:102D10000000000000808080808080800000000033
:102D200000000000000000000000000000000000A3
:102D3000000000000000000000000000003FFFFF56
:102D4000FFFFFFFC00C0FFFFFFFF7FFFFFFFFFFF54
:102D50008000FEFFFFFFFFFF0F000000F0F8FEFE07
:102D6000FFFF7F1F0F0F1FFFFFFFFEFCF8C00000DB
:102D70000000C0FCFFFFFFFF7F071FFFFFFFFFFFFB
:102D8000F88000000000C0F0FCFEFFFFFF7F1F1F67
:102D90001F1F3F3F3F0E041F1FFFFFFFFFFFFFFFEF
:102DA0001F1F1F1F000000000000000000000000A7
:102DB0001F7FFFFFFFFFFFFCF8F8F0F0E0E0C1C06D
:102DC0008000001F1F1FFFFFFFFFFFFFFF1F1F1FD0
:102DD0000F000000FFFFFFFFFFFF00000000FFFFEC
:102DE000FFFFFFFFFF000000C0F8FCFEFFFFFF7FBA
:102DF0001F1F1F3FFFFFFFFFFFFFFF00000000FF3F
:102E0000FFFFFFFFFFFF000000C0F8FCFEFFFFFF19
:102E10003F1F1F1F3FFFFFFFFEFCF8E00000000008
:102E200000000000000000000000000000000000A2
:102E300000000000000000000FFFFFFFFFFFFCFF8D
:102E4000FFFFFF1F0001FFFFFFFFFFFEFFFFFFFF70
:102E5000FF070000001EFFFFFFFFFFFFDF1F1F1F18
:102E60001F1F1F9F9F1F1F1F0000E0FEFFFFFFFF90
:102E7000FFFFFCFCFCFDFFFFFFFFFFFFFCC00000AD
:102E8000FFFFFFFFFFFFFF80000000000080000049
:102E9000000000FFFFFFFFFFFFFF00000000000039
:102EA0000000000000000000000080C0C0800101A0
:102EB000030303070FFFFFFFFFFFFFFF700000008A
:102EC000FFFFFFFFFFFFFF00000000000000FFFF0B
:102ED000FFFFFFFF00000080FFFFFFFFFFFFFF007D
:102EE0000000FFFFFFFFFFFFFF8000000000FFFF6B
:102EF000FFFFFFFFFF00000000FFFFFFFFFFFFFFDE
:102F0000000000FFFFFFFFFFFFFF8000000000FF49
:102F1000FFFFFFFFFFFF00000000000000000000B7
:102F200000000000000000000000000000000000A1
:102F3000000000073F3F3F3F3F3F3F3F0F00000083
:102F4000003F3F3F3F3F3F3F3F3F01000000000049
:102F500001070F1F1F3F3F3F3E3E3E3E3F3F1F1FAB
:102F60000E00303E3F3F3F3F3F1F0100000000008A
:102F700000033F3F3F3F3F3F3C000003070F1F3F21
:102F80003F3F3F3E3E3F3F3F1F1E080000030F1FD5
:102F90003F3F3F3F3F3E3F3F1C1800000000000006
:102FA000000000070F1F1F3F3F3F3F3E3E3F3F3F98
:102FB0003F1F1F0F070300000000070F1F3F3F3F89
:102FC0003F3E3F3F3F1C00000F1F3F3F3F3F3F3E04
:102FD0003F1F1F3F3F3F3F3F3F00000000070F1FC5
:102FE0003F3F3F3F3F3E3F1F1F3F3F3F3F3F3F0071
:102FF0000000003F3F3F3F3F3F3F0000000003070E
:103000000F1F3F3F3F3F3E3E3F3F3F1F1F0F03000D
:1030100000000000000000000000000000000000B0
:1030200000000000000000000000000000000000A0
:103030000000000000000000000000000000000090
:103040000000000000000000000000000000000080
:103720000000000000000000C0C0C0C0C000008059
:10373000C0C0C0C080000000000000000000000009
:103740000000000000000000000000000000000079
:103750000000000000000000000000000000000069
:103760000000000000000000000000000000000059
:103770000000000000000000000000000000000049
:103780000000000000000000000000000000000039
:103790000000000000000000000000000000000029
:1037A0000000000000000000000000000000000019
:1037B0000000000000000000000000C0C0C0C0C049
:1037C000C000000000000000000000000000000039
:1037D00000C0C0C0C0C00000000000000000000029
:1037E00000000000000000000000000000000000D9
:1037F00000000000000C1E1F1F0F0F9FFFFFFEFEAA
:10380000F80000000000000038787C7E3EFFFFFFDB
:10381000FFFF00040E1E1F8F8F8FFFFFFFFEFC00B7
:103820000000737F3F1F0F0000317B7F3F1F0700A9
:1038300000000000000000FFFFFFFFFF8787878771
:1038400087070000F0F0F0F0F0F070F8F8F0F0E02A
:10385000800030F0F0F07878F8F0F0F0E0800000D0
:10386000F0F0F0F0F0F070F8F8F0F0E0800080E0B8
:10387000F0F0F0F878F0F0F0E0C00000F0F0F0F0D8
:10388000F0F0F0F0F01000000000000000FFFFFF7B
:10389000FFFFFFFEC0E0FFFFFFFFFFFFFF00008014
:1038A000C0E0F0F0F078F8F0F0F0E0C00000C0E028
:1038B000F0F0F8F870FFFFFFFFFFFF0000F0F0F0FE
:1038C000F0F000F0F0F0F0F0F00000FFFFFFFFFF7D
:1038D000000080C0E0F0F0F878F8F0F0F0E0800050
:1038E0000000000000000000000000000000008058
:1038F000C0F0F8FCFEFFBF9F87838000C0C0C0C03F
:10390000C0800000000000FFFFFFFFFF0080C0C07C
:10391000C0C78787CFFFFFFFFEF800000000000050
:103920000000000000000000000000000000000097
:1039300000FFFFFFFFFF8787878787800000FFFF6B
:10394000FFFFFF8080E1FFFFFFFF7F40F8FCFCFEF0
:10395000FE9ECFFFFFFFFFFF0000FFFFFFFFFF8086
:1039600080E1FFFFFFFF7F00FFFFFFFFFFDC9C9D6B
:103970009FDFDF9F1F00FFFFFFFFFF03010000002D
:10398000000000000000FFFFFFFFFF0FFFFFFFFF31
:10399000FFFF0FFFFFFFFFFC007FFFFFFFFFE18046
:1039A00080FFFFFFFFFF1C08FFFFFFFFFF8080FF7E
:1039B000FFFFFFFFFF0000FFFFFFFFFF80FFFFFF94
:1039C000FFFFFF0000FFFFFFFFFF80007FFFFFFF03
:1039D000FFDC9C9C9FDFDF9F1F00000000000000B9
:1039E00000000000000000000007070707070707A6
:1039F0000707070707000307070707030000000082
:103A00000007070707070001030307070707070762
:103A1000070301000000000000000000000000009B
:103A20000000000000000000000000070707070773
:103A30000707070707070000FFFFFFFFFF0707074C
:103A40000707030100000307070707070703070726
:103A500007070000FFFFFFFFFF0707070707030136
:103A6000000000010307070707070707030300001B
:103A70000707070707000000000000000000000023
:103A800007070707070001010101010000070707F9
:103A900007070000010307070707070707030300DD
:103AA00000000103070707070707070707070700C5
:103AB00000030707070707070707070707000003B3
:103AC0000707070707070001030707070707070797
:103AD00003030000000000000000000000000000E0
:103AE00000000000000000000000000000000000D6
:103AF00000000000000000000000000000000000C6
:103B000000000000000000000000000000000000B5
:103B100000000000000000000000000000000000A5
:1040E00000000000000000000000000070F0F8FC7C
:1040F0007CFEFEFEFEFE00183C3C3E3E1E1EFEFE0A
:10410000FEFCF800183C3E3E1E1E3EFEFEFCFCF08F
:1041100000000000000000E0E0E0E0E0C080E0E03F
:10412000E0E0E0000000000000183C3C3E3E1E1EA7
:10413000FEFEFEFCF80000FEFEFEFEFE9E9E9E9E23
:104140001E1E0000E0F8FCFEFE7E1E3EFEFEFCF899
:10415000E00000000000000000FEFEFEFEFEFE0E7D
:104160000E0E0E0E0E000000000000000000000009
:1041700000FEFEFEFEFE00000000000000FEFEFE4F
:10418000FEFE000000FEFEFEFEFEFEFCE000FEFE67
:10419000FEFEFE0000FEFEFEFEFEC0E0F8FCFEFE9F
:1041A0003E1E0600000000000000000000000000AD
:1041B00000000000000000000000000000000000FF
:1041C00000000000000000000000000000000000EF
:1041D00000000000000000000000000000000000DF
:1041E0000000000000000000000000FFFFFFFFFFD4
:1041F000000080C0E0F0FCFE7F3F1F0F0300008046
:10420000E0F0F8FCFF7F3F0F070100000000000016
:104210000000C1E7FFFFFFFFFFFFF7C10000000044
:104220000000000080C0E0F0FCFE7F3F1F0F030095
:10423000008787878707078FFFFFFFFFFC007FFF4F
:10424000FFFFFFC00080FFFFFFFFFF000000000036
:10425000000000FFFFFFFFFFFF0F0F0F0F0F000019
:104260001E1E1E1E1E1E1E1E1E0000FFFFFFFFFF45
:1042700000000000000000FFFFFFFFFF000000FF44
:10428000FFFFFFFF3FFFFFFFFFFFFFFFFF0000FFFC
:10429000FFFFFFFF1F7FFFFFFFF8E0C000000000EF
:1042A000000000000000000000000000000000000E
:1042B00000000000000000000000000000000000FE
:1042C00000000000000000000000000000000000EE
:1042D00000000000000000000000000000000000DE
:1042E00000000000000F0F0F0F0F00000F0F0F0F47
:1042F0000F0F0F0F0F0F0F070F0F0F0F0F0F0F0FD6
:104300000F0F0F0F0000000000000C0F0F0F0F0F1A
:104310000101070F0F0F0F0C0000000000000F0F2E
:104320000F0F0F0F0F0F0F0F0F070307070F0F0FC1
:104330000F0F0F0F070301000003070F0F0F0F0FE1
:104340000F0F07030000000000000000000F0F0F18
:104350000F0F0F0F0F0F0F0F0F00000000000000D6
:1043600000000000000F0F0F0F0F0F0F0F0F0F0FA8
:10437000000F0F0F0F0F0000000F0F0F0F0F0001A6
:104380000F0F0F0F0F0F0F00000F0F0F0F0F000079
:1043900001030F0F0F0F0F0C0000000000000000C2
:1043A000000000000000000000000000000000000D
:1043B00000000000000000000000000000000000FD
:1043C00000000000000000000000000000000000ED
:1043D00000000000000000000000000000000000DD
:1043E00000000000000000000000000000000000CD
:1043F00000000000000000000000000000000000BD
:1044000000000000000000000000000000000000AC
:10441000000000000000000000000000000000009C
:10442000000000000000000000000000000000008C
:10443000000000000000000000000000000000007C
:10444000000000000000000000000000000000006C
:10445000000000000000000000000000000000005C
:10446000000000000000000000000000000000004C
:10447000000000000000000000000000000000003C
:10448000000000000000000000000000000000002C
:10449000000000000000000000000000000000001C
:1044A000000000000000000000000000000000000C
:1044B00000000000000000000000000000000000FC
:1044C00000000000000000000000000000000000EC
:1044D00000000000000000000000000000000000DC
:1044E00000000000000000000000000000000000CC
:1044F00000000000000000000000000000000000BC
:1045000000000000000000000000000000000000AB
:10451000000000000000000000000000000000009B
:10452000000000000000000000000000000000008B
:10453000000000000000000000000000000000007B
:10454000000000000000000000000000000000006B
:10455000000000000000000000000000000000005B
:10456000000000000000000000000000000000004B
:10457000000000000000000000000000000000003B
:10458000000000000000000000000000000000002B
:10459000000000000000000000000000000000001B
:1045A000002F000000000700070000147F147F1494
:1045B00000242A7F2A12006264081323003649551A
:1045C000225000000503000000001C2241000000F2
:1045D00041221C000014083E08140008083E080888
:1045E000000000A0600000080808080800006060E3
:1045F0000000002010080402003E5149453E000022
:10460000427F4000004261514946002141454B3103
:10461000001814127F10002745454539003C4A49CF
:104620004930000171090503003649494936000641
:104630004949291E000036360000000056360000A9
:104640000008142241000014141414140000412224
:10465000140800020151090600324959513E007CFC
:104660001211127C007F49494936003E41414122E6
:10467000007F4141221C007F49494941007F0909CF
:104680000901003E4149497A007F0808087F00007F
:10469000417F4100002040413F01007F081422413A
:1046A000007F40404040007F020C027F007F0408F2
:1046B000107F003E4141413E007F09090906003E4E
:1046C0004151215E007F0919294600464949493177
:1046D0000001017F0101003F4040403F001F20409A
:1046E000201F003F4038403F006314081463000758
:1046F0000870080700615149454300007F414100AF
:1047000000552A552A55000041417F00000402014E
:10471000020400404040404000000102040000202C
:1047200054545478007F484444380038444444206A
:1047300000384444487F00385454541800087E0917
:1047400001020018A4A4A47C007F080404780000DF
:10475000447D4000004080847D00007F102844009C
:104760000000417F4000007C04180478007C0804AD
:10477000047800384444443800FC242424180018E9
:10478000242418FC007C08040408004854545420D5
:1047900000043F444020003C4040207C001C20405E
:1047A000201C003C4030403C004428102844001CA1
:1047B000A0A0A07C004464544C4414141414141499
:1047C0000000000000000000000000000000FC00ED
:1047D0000000000002000000000C020C02000000BB
:1047E0000000000090D0BCD0BC900003000300008B
:1047F0001824FE448C000302070201001824D8B0DC
:104800004C80000300010201C038E438E0000102DE
:104810000201020208060000000000000000000083
:10482000000000F80402000000010204000204F885
:1048300000000004020100009060F8609000000099
:10484000010000002020FC202000000001000000EA
:1048500000000000000008060000000020202020CA
:104860002000000000000000000000000000000226
:10487000000000000080601C020004030000000033
:10488000F8040404F8000102020201000008FC0020
:1048900000000002030200001884442418000302F0
:1048A0000202020008042424D800010202020100CE
:1048B00040B088FC80000000000302003C24242457
:1048C000C400010202020100F824242CC0000102ED
:1048D000020201000C04E41C0400000003000000BC
:1048E000D8242424D80001020202010038444444A0
:1048F000F8000003020201000000100000000000A8
:10490000020000000000200000000000060000007F
:104910000020508804020000000001029090909056
:1049200090000000000000000002048850200002F7
:10493000010000001804C424180000000200000058
:10494000F804E494F80001020202020000E09CF086
:10495000800002030000030204FC2424D8000203A8
:1049600002020100F80404040C000102020201002A
:1049700004FC0404F80002030202010004FC247495
:104980000C0002030202030004FC24740C00020366
:1049900002000000F0080444CC40000102020100C3
:1049A00004FC2020FC040203000003020404FC04B5
:1049B0000400020203020200000404FC04040604D2
:1049C0000403000004FC24D00C04020302000302D0
:1049D00004FC04000000020302020203FC3CC03C91
:1049E000FC0003000300030004FC30C4FC040203C9
:1049F00002000300F8040404F800010202020100AE
:104A000004FC24241800020302000000F88484043B
:104A1000F80001020207050004FC24649800020368
:104A200002000302182424448C0003020202010045
:104A30000C04FC040C0000020302000004FC000053
:104A4000FC04000102020100047C80E01C04000060
:104A5000030000001CE03CE01C0000030003000019
:104A6000049C609C0400020300030200041CE01C80
:104A700004000002030200000C84641C0400020312
:104A8000020203000000FE0202000000070404000E
:104A9000000E30C00000000000010200000202FE13
:104AA00000000004040700000004020400000000ED
:104AB00000000000000000000000080808080808C6
:104AC0000000020000000000000000000040A0A064
:104AD000C00000010202030204FC2020C000000309
:104AE0000202010000C0202060000001020202005A
:104AF00000C02024FC0000010202030200C0A0A0AC
:104B0000C0000001020202000020F8242404000278
:104B1000030202000040A0A0602000070A0A0A0465
:104B200004FC2020C0000203020003020020E40075
:104B30000000000203020000000020E4000008085A
:104B40000807000004FC80E02020020302000302AA
:104B50000404FC000000020203020200E020E02046
:104B6000C00003000300030020E02020C000020377
:104B70000200030200C02020C00000010202010068
:104B800020E02020C000080F0A02010000C0202001
:104B9000E0000001020A0F0820E04020200002038C
:104BA000020000000060A0A020000002020203003A
:104BB0000020F820000000000102020020E0002098
:104BC000E00000010202030220E0208060200000DB
:104BD000030100006080E08060000003000300002B
:104BE00020608060200002030003020020E020809B
:104BF00060200808070100000020A06020000002DB
:104C000003020200000020DE020000000007040092
:104C1000000000FF00000000000F00000002DE2086
:104C2000000000040700000002010204040200006A
:104C30000000000000000000000000000000000074
:104C400000000000000000F8000000000000003339
:104C50003000000000100C06100C060000000000E0
:104C60000000000040C07840C0784000043F0404C9
:104C70003F040400007088FC08300000001820FF8A
:104C8000211E0000F008F000E018000000211C03C5
:104C90001E211E0000F00888700000001E21232441
:104CA0001927211010160E0000000000000000005F
:104CB00000000000000000E01804020000000007EF
:104CC0001820400000020418E000000000402018F6
:104CD00007000000404080F0804040000202010FC9
:104CE00001020200000000F0000000000101011FAD
:104CF00001010100000000000000000080B0700011
:104D000000000000000000000000000000010101A0
:104D1000010101010000000000000000003030002F
:104D20000000000000000000806018040060180609
:104D30000100000000E010080810E000000F102043
:104D400020100F00001010F8000000000020203F8D
:104D50002020000000700808088870000030282417
:104D600022213000003008888848300000182020B8
:104D700020110E000000C02010F8000000070424DD
:104D8000243F240000F80888880808000019212022
:104D900020110E0000E0108888180000000F11207C
:104DA00020110E0000380808C83808000000003F35
:104DB000000000000070880808887000001C222194
:104DC00021221C0000E010080810E0000000312241
:104DD00022110F00000000C0C000000000000030E1
:104DE0003000000000000080000000000000806033
:104DF00000000000000080402010080000010204B4
:104E0000081020004040404040404000040404049A
:104E10000404040000081020408000000020100856
:104E200004020100007048080808F000000000308B
:104E300036010000C030C828E810E0000718272419
:104E400023140B000000C038E0000000203C2302C7
:104E50000227382008F8888888700000203F20202A
:104E600020110E00C030080808083800071820205C
:104E70002010080008F808080810E000203F202053
:104E800020100F0008F88888E8081000203F202034
:104E90002320180008F88888E8081000203F200028
:104EA00003000000C0300808083800000718202060
:104EB000221E020008F808000008F808203F21011F
:104EC00001213F20000808F8080800000020203FCA
:104ED0002020000000000808F8080800C08080803A
:104EE0007F00000008F888C028180800203F200133
:104EF0002638200008F8080000000000203F20208D
:104F00002020300008F8F800F8F80800203F003FA3
:104F1000003F200008F830C00008F808203F2000BB
:104F200007183F00E01008080810E0000F102020CC
:104F300020100F0008F808080808F000203F2101A1
:104F400001010000E01008080810E0000F182424F8
:104F500038504F0008F8888888887000203F20006B
:104F6000030C302000708808080838000038202121
:104F700021221C00180808F8080818000000203F2B
:104F80002000000008F808000008F808001F202092
:104F900020201F000878880000C838080000073863
:104FA0000E010000F80800F80008F800033C0700B4
:104FB000073C0300081868808068180820302C031C
:104FC000032C30200838C800C83808000000203FF3
:104FD0002000000010080808C838080020382621E2
:104FE00020201800000000FE020202000000007FE6
:104FF00040404000000C30C00000000000000001F4
:105000000638C00000020202FE00000000404040DE
:105010007F00000000000402020204000000000003
:105020000000000000000000000000008080808080
:105030008080808000020204000000000000000068
:105040000000000000008080808000000019242201
:1050500022223F2008F8008080000000003F11203D
:1050600020110E000000008080800000000E112042
:1050700020201100000000808088F800000E112020
:1050800020103F200000808080800000001F22222E
:1050900022221300008080F0888888180020203F9A
:1050A000202000000000808080808000006B9494AD
:1050B0009493600008F8008080800000203F210069
:1050C00000203F2000809898000000000020203F32
:1050D00020200000000000809898000000C0808020
:1050E000807F000008F8000080808000203F2402BC
:1050F0002D302000000808F8000000000020203FAC
:10510000202000008080808080808000203F200060
:105110003F20003F8080008080800000203F2100F1
:1051200000203F200000808080800000001F2020A1
:1051300020201F00808000808000000080FFA120D0
:1051400020110E000000008080808000000E1120E1
:1051500020A0FF80808080008080800020203F2170
:105160002000010000008080808080000033242423
:1051700024241900008080E0808000000000001FCF
:10518000202000008080000000808000001F202080
:1051900020103F20808080000080808000010E3041
:1051A0000806010080800080008080800F300C03A2
:1051B0000C300F0000808000808080000020312EA5
:1051C0000E312000808080000080808080818E7081
:1051D0001806010000808080808080000021302C33
:1051E0002221300000000000807C0202000000004C
:1051F000003F404000000000FF00000000000000F1
:10520000FF0000000002027C800000000040403FE0
:10521000000000000006010102020404000000007A
:10522000000000000000000000000000000000007E
:10523000000000000000000000000000000000006E
:1052400000000000000000000000000000F0F0F08E
:10525000000000000000000000017F0100000000CD
:1052600000000000001C1C1C00000000000080600A
:10527000301C8C60301C0C0000000000000000009E
:10528000000000000000000000000000000000001E
:10529000000000E00000000000E000000086E69F43
:1052A00086868686E69F860000011F0101010101B6
:1052B0001F010100000080C06020F820E0C0000055
:1052C000000003070C18FF70E18100000000070FC9
:1052D00010107F100F070000806020608000000029
:1052E000E02000000F3020309F70DC371030C0000D
:1052F0000000100E03000718101807000000C0205F
:1053000020E0C0000000000080E01F38E88703C4F0
:105310003C040000070F1810100B070D10100800B8
:1053200000808C4C380000000000000000000000ED
:10533000000000000000000000000000000000006D
:105340000000000000000000000080E030080400C1
:105350000000000000FEFF0100000000000000004F
:105360000000030F1820400000040830E080000017
:10537000000000000000000001FFFE00000000002F
:10538000004020180F030000000000000000000093
:105390000000C00000000000004266663C18FF18D4
:1053A0003C666642000000000000030000000000B0
:1053B000000000000000800000000000001010103D
:1053C0001010FF101010101000000000000003006B
:1053D00000000000000000000000000000000000CD
:1053E00000000000000000000000000000808C4C65
:1053F0003800000000000000000000000000000075
:1054000000000000001010101010101010101000FC
:10541000000000000000000000000000000000008C
:10542000000000000000000000000000000000007C
:105430000000000000001C1C1C0000000000000018
:105440000000000000000000E0380C000000000038
:1054500080701C03000000000060380E0100000096
:1054600000000000000080C060202060C0800000BC
:1054700000FEFF010000000001FFFE000001070E1A
:10548000181010180E0701000000808080C0E00096
:10549000000000000000000000FFFF00000000000E
:1054A00000001010101F1F1010100000008040207E
:1054B00020202060C08000000003030080402038CE
:1054C0001F070000001C1A1918181818181F0000D0
:1054D0000080C020202060C0800000000003030086
:1054E0001010182FE780000000070F101010101880
:1054F0000F070000000000000000C0E0F000000006
:1055000000C0B088868180FFFF808000000000001E
:105510000010101F1F1010000000E060606060604D
:105520006060000000003F1008080818F0E000006C
:1055300000070B101010101C0F030000000080C0AB
:1055400040202020E0C0000000FCFF2110080808D7
:1055500018F0E0000001070C18101010080F0300ED
:105560000000C0E06060606060E060000000030078
:105570000000E0180700000000000000001F1F00EE
:10558000000000000080C0602020202060C080005B
:105590000087EF2C1818303068CF830000070F0801
:1055A00010101010180F07000000C0C0202020208D
:1055B000C0800000001F3F604040402010FFFE0000
:1055C00000000C1C101010080F0300000000000069
:1055D000000000000000000000000000000E0E0EA1
:1055E0000000000000000000001C1C1C0000000067
:1055F00000000000000000000000000000000000AB
:10560000000C0C00000000000000000000583800F2
:10561000000000000000000000000080402010009A
:10562000000010284482010000000000000000007B
:10563000000001020408100000000000000000004B
:105640000000000000848484848484848484840032
:10565000000000000000000000000000000010201A
:1056600040800000000000000000000000000182F7
:10567000442810000000100804020100000000008F
:1056800000C020201010101030E0C0000003030004
:1056900000F010080C070300000000001C1C1C0098
:1056A00000000000000000C0406020202040C0003A
:1056B00000FCFF01F00E03C1FE03807F0001070E16
:1056C00008111110110904020000000080E0E00040
:1056D000000000000000807C4340477FF88000000D
:1056E00010181F1000000000131F1C1020E0E02005
:1056F00020202060C080000000FFFF101010101854
:105700002FE78000101F1F1010101010180F070037
:10571000000080C0402020202060E00000FCFF014D
:1057200000000000000001000001070E181010101A
:105730000804030020E0E02020202040C08000007A
:1057400000FFFF000000000001FFFE00101F1F10FF
:10575000101018080E07010020E0E0202020202073
:105760002060800000FFFF101010107C000000007F
:10577000101F1F10101010101018060020E0E0205D
:10578000202020206060800000FFFF101010107C9F
:1057900000000100101F1F100000000000000000AA
:1057A000000080C06020202040E0000000FCFF01DD
:1057B00000004040C0C140400001070E181010100A
:1057C0000F0F000020E0E0200000000020E0E020BB
:1057D00000FFFF101010101010FFFF00101F1F100F
:1057E00000000000101F1F100000202020E0E0201B
:1057F000202000000000000000FFFF00000000006B
:1058000000001010101F1F101010000000000000FA
:10581000202020E0E020202000000000000000FF09
:10582000FF0000000060E0808080C07F3F0000003B
:1058300020E0E020000020A06020200000FFFF30DA
:10584000187CE3C000000000101F1F1000000113AF
:105850001F1C181020E0E0200000000000000000E5
:1058600000FFFF000000000000000000101F1F10DC
:10587000101010101018060020E0E0E000000000FA
:10588000E0E0E02000FF013FFEC0E01E01FFFF005E
:10589000101F1000031F0300101F1F1020E0E0C0A6
:1058A000000000000020E02000FF0003071C78E05B
:1058B0008000FF00101F100000000000030F1F00F9
:1058C000000080C060202060C080000000FEFF015A
:1058D0000000000000FFFE000001070E1810101865
:1058E0000C07010020E0E0202020202060C0800084
:1058F00000FFFF2020202020301F0F00101F1F104E
:105900000000000000000000000080C06020206057
:10591000C080000000FEFF010000000000FFFE004C
:105920000001070E1111133C7C67210020E0E020EC
:105930002020202060C0800000FFFF101030F0D039
:10594000080F0700101F1F10000000030F1C10108D
:105950000080C060202020204040E00000070F0CA5
:105960001818303060E08100001F0C081010101073
:10597000180F07008060202020E0E02020206080B9
:105980000100000000FFFF00000000010000000017
:10599000101F1F100000000020E0E02000000000A9
:1059A0000020E02000FFFF00000000000000FF00DA
:1059B00000070F1810101010100807002060E0E01A
:1059C0002000000020E060200000077FF8800080B9
:1059D0007C03000000000000071F1C0700000000FF
:1059E00020E0E02000E0E0200020E0200007FFF8B9
:1059F000E01FFFFCE01F00000000031F0300011F69
:105A000003000000002060E0A0000020E060200013
:105A1000000000038F7CF8C6010000000010181E73
:105A2000130001171F1810002060E0E020000000A4
:105A300020E06020000001073EF8E01807000000A9
:105A400000000010101F1F101000000000806020D8
:105A5000202020A0E0E0200000000000C0F03E0F69
:105A60000300000000101C1F171010101018060073
:105A70000000000000FC0404040404000000000016
:105A800000FF00000000000000000000007F404018
:105A900040404000000010E0000000000000000056
:105AA00000000000031C60800000000000000000F7
:105AB000000000030C70800000000404040404FCD7
:105AC0000000000000000000000000FF00000000D7
:105AD000000040404040407F0000000000000010F7
:105AE000080C040C0810000000000000000000007A
:105AF00000000000000000000000000000000000A6
:105B00000000000000000000000000000000000095
:105B10000000000000000000808080808080808085
:105B2000808080800000000404080800000000005D
:105B30000000000000000000000000000000000065
:105B40000000000000000000000000000000000055
:105B500000000000000098D844642424FCF80000F1
:105B6000000F1F18101010081F1F10180020E0F061
:105B700000000000000000000000FFFF18080404FF
:105B80000CF8F00000001F0F18101010180F030081
:105B900000000000000000000000000000E0F81815
:105BA0000404043C3800000000030F0C1010101017
:105BB000080600000000000000000020E0F00000E7
:105BC00000E0F81C04040408FFFF000000030F18A5
:105BD000101010081F0F0800000000000000000057
:105BE000000000000000E0F8484444444C78700095
:105BF0000000030F0C181010100804000000000033
:105C000080C0602020E0C00000040404FFFF040402
:105C100004040000000010101F1F101010000000EE
:105C2000000000000000000000000000000070F80C
:105C30008C04048CF874040C007076CF8D8D8D89E3
:105C4000C87870000020E0F00000000000000000B4
:105C50000000FFFF08040404FCF8000000101F1FF0
:105C6000100000101F1F1000000000000060600006
:105C7000000000000000040404FCFC000000000020
:105C800000001010101F1F10101000000000000076
:105C9000000000606000000000000000040404FC3C
:105CA000FC0000000000C0C08080C07F3F000000FA
:105CB0000020E0F000000000000000000000FFFFF6
:105CC00080C0F41C0404000000101F1F1100031FFB
:105CD0001C1010000000202020E0F0000000000058
:105CE0000000000000FFFF00000000000000101096
:105CF000101F1F1010100000000000000000000026
:105D00000000000004FCFC0804FCFC0804FCFC008F
:105D1000101F1F10001F1F10001F1F100000000089
:105D200000000000000000000004FCFC080804045F
:105D3000FCF8000000101F1F100000101F1F1000B3
:105D400000000000000000000000000000E0F0186B
:105D50000C04040C18F0E00000030F0C10101010DD
:105D60000C0F030000000000000000000000000015
:105D70000004FCFC080404040CF8F0000080FFFFA1
:105D8000889010101C0F03000000000000000000AD
:105D90000000000000E0F81C04040408F8FC000007
:105DA00000030F1810109088FFFF80000000000013
:105DB0000000000000000000040404FCFC100804C3
:105DC000040C0C001010101F1F1010100000000019
:105DD000000000000000000000000000000030781B
:105DE000CCC48484840C1C0000001E1810101011F8
:105DF000190F06000000000000C0000000000000B5
:105E000000040404FFFF040404000000000000007C
:105E10000F1F1010100C0000000000000000000018
:105E2000000000000004FCFE00000004FCFE000076
:105E300000000F1F181010081F0F080000000000BE
:105E4000000000000000000000040C3CFCC4000046
:105E5000C43C0C0400000000010F1E0E01000000F5
:105E6000000000000000000000000000043CFCC432
:105E700000E47CFC84807C040000071F070000070E
:105E80001F070000000000000000000000000000EC
:105E90000004041C7CE4C0341C0404000010101C2A
:105EA0001601131F1C181000000000000000000065
:105EB0000000000000040C3CFCC400C43C040400CE
:105EC0000000C080C1370E0100000000000000008B
:105ED000000000000000000000001C0404C4F47C6A
:105EE0001C0400000000101C1F17111010180E00D9
:105EF00000000000000000F80C040000000000009A
:105F0000001028EF00000000000000000000003F2B
:105F100060400000000000000000FF0000000000E2
:105F2000000000000000FF00000000000000000072
:105F30000000FF00000000000000040CF80000005A
:105F40000000000000000000EF281000000000002A
:105F5000000040603F000000000000000018060242
:105F6000020408102020300800000000000000009B
:105F70000000000000000000000000000000000021
:105F80000000F010101010FF10101010F0000000B2
:105F900000000F04040404FF040404040F000000C4
:105FA0004040405F555555755555555F4040400040
:105FB0000040200F094989790909090F2040000094
:105FC00000FE02424ACA4A4ACA4A4A4202FE000047
:105FD00000FF40504C4340404F50505C40FF000099
:105FE0000000F888888888FF88888888F800000082
:105FF00000001F080808087F888888889F80F000B4
:1060000080828282828282E2A2928A86828080005C
:10601000000000000040807F000000000000000041
:10602000101010FF109008888888FF888888080062
:106030000444827F01808040432C102846818000E8
:106040000010101010D030FF30D0121C10100000C3
:1060500010080402010000FF000001020408100003
:1060600004040484E43C2724242424E404040400D9
:1060700004020100FF0909090949897F00000000A5
:1060800000FE225A8600FE9292929292FE0000003A
:1060900000FF04080700FF4020030C1422414000C9
:1060A0000080402018068000071820408000000073
:1060B00001002070282621202024386000010100E2
:1060C000001012929292929292121202FE0000001E
:1060D0000000003F101010103F0040807F000000C3
:1060E000000000C080808080808080FC8480808070
:1060F000808080C0C0000000000000FF7F40404062
:10610000404040FF40404040404040FF7F00000092
:1061100000000000000000000000007F7000000090
:10612000000000000000000000000000000000006F
:1061300000000000000000FCF8000000000000006B
:10614000000000000000000000000000FFFE02024E
:1061500002020202020202FFFF0202020202020225
:106160000202FF0300000000000000001F1F0404E3
:1061700004040404040404FFFF04040404040404E9
:1061800004041F00000000000000000000000000E8
:10619000000000000000007F3F0000000000000041
:1061A00000000000000000000000000000000000EF
:1061B00000000000000000000000000000000000DF
:1061C0000000000000F8F8F0F0702000000000006F
:1061D00000000000000000000000000000000000BF
:1061E00000000000000000000000000000000000AF
:1061F000800000000000000000000000000000001F
:106200000000000000FFFFFFFF0000000000000092
:10621000000000000000000000000000808000007E
:10622000000000000000000000000000000000006E
:1062300000FFFFFE0606060606060606060606061A
:106240000606060606FFFFFFFF060606060606060A
:106250000606060606060606060606FFFFFFFF07F9
:10626000020000000000000000000000000000002C
:1062700000FFFFFF00000000000000000000000021
:106280000000000000FFFFFFFF0000000000000012
:106290000000000000000000000000FFFFFFFF0002
:1062A00000000000000000000000000000000000EE
:1062B00000FFFFFF181818181818181818181818C1
:1062C0001818181818FFFFFFFF18181818181818B2
:1062D0001818181818181818181818FFFFFFFF00BA
:1062E00000000000000000000000000000000000AE
:1062F000020101000000000000000000000000009A
:106300000000000000FFFFFFFF0000000000000091
:10631000000000000000000000000001010000007B
:10632000000000000000000000000000000000006D
:10633000000000000000000000000000000000005D
:106340000000000000FFFFFFFF0000000000000051
:10635000000000000000000000000000000000003D
:10636000000000000000000000000000000000002D
:10637000000000000000000000000000000000001D
:1063800000000000001F1F0F0F00000000000000B1
:1063900000000000000000000000000000000000FD
:1063A0000000000000000000C8630008000000209A
:1063B0001C000000AC070008E46300081C0000207B
:1063C00054230000BC07000800000000000000008B
:1063D000000000000000000000000000000E270781
:0463E00000000000B9
:0400000508000131BD
:00000001FF
